:020000040800F2
:10000000301A00208901000839420008E93F000841
:100010003542000815030008AD610008000000002B
:10002000000000000000000000000000F95C000873
:100030001505000800000000594C0008515D00083B
:10004000A3010008A3010008A3010008A301000800
:10005000A3010008A3010008A3010008A3010008F0
:10006000A3010008A3010008A3010008A3010008E0
:10007000A3010008A3010008A3010008A3010008D0
:10008000A3010008A3010008A30100088D61000876
:100090009D6100081903000829030008A301000856
:1000A000A3010008A3010008A3010008A3010008A0
:1000B000A3010008A3010008F95D0008A3010008DE
:1000C000A3010008A3010008A3010008A301000880
:1000D000A3010008A3010008A3010008A301000870
:1000E000A3010008A3010008A301000800F002F822
:1000F00000F03AF80AA090E8000C82448344AAF188
:100100000107DA4501D100F02FF8AFF2090EBAE885
:100110000F0013F0010F18BFFB1A43F0010318473B
:10012000A8620000C8620000103A24BF78C878C1F5
:10013000FAD8520724BF30C830C144BF04680C60ED
:10014000704700000023002400250026103A28BF35
:1001500078C1FBD8520728BF30C148BF0B60704739
:100160001FB51FBD10B510BD00F08AF81146FFF78E
:10017000F7FF06F0ADF800F0A8F803B4FFF7F2FFC0
:1001800003BC00F0AFF80000094880470948004769
:10019000FEE7FEE7FEE7FEE7FEE7FEE7FEE7FEE737
:1001A000FEE7FEE704480549054A064B7047000094
:1001B000F55D0008ED00000830140020301A002022
:1001C000301600203016002010B5203AC0F00B8009
:1001D000B1E81850A0E81850B1E81850A0E818503D
:1001E000203ABFF4F5AF5FEA027C24BFB1E81850B3
:1001F000A0E8185044BF18C918C0BDE810405FEA15
:10020000827C24BF51F8043B40F8043B08BF704790
:10021000D20728BF31F8023B48BF11F8012B28BF95
:1002200020F8023B48BF00F8012B70474FF0000256
:1002300000B5134694469646203922BFA0E80C50DC
:10024000A0E80C50B1F12001BFF4F7AF090728BFB7
:10025000A0E80C5048BF0CC05DF804EB890028BF33
:1002600040F8042B08BF704748BF20F8022B11F05C
:10027000804F18BF00F8012B7047704770477047D8
:10028000754600F02BF8AE4605006946534620F04F
:100290000700854618B020B5FFF784FFBDE8204071
:1002A0004FF000064FF000074FF000084FF0000B32
:1002B000AC46ACE8C009ACE8C009ACE8C009ACE8A1
:1002C000C00921F007018D46704710B50446AFF311
:1002D00000802046BDE81040FFF74FBF0048704740
:1002E0002800002001491820ABBEFEE726000200CE
:1002F0007047000040F6E400C2F20000007840F2CF
:100300000001C2F200010978401A813000F07F003C
:1003100070470000FFE7FEE780B540F6FC00C2F240
:10032000000000F06FFC80BD80B540F6FC00C2F21A
:10033000000000F067FC80BD40F28801C2F20001BD
:10034000486901304861704740F28801C2F20001FB
:10035000C8690130C861704740F28801C2F20001EB
:10036000886801308860704740F28801C2F200015D
:10037000886901308861704740F28801C2F200014B
:10038000086A01300862704740F28801C2F2000139
:10039000486801304860704740F28801C2F20001AD
:1003A000086801300860704740F28801C2F200011D
:1003B000086901300861704740F28801C2F200010B
:1003C000886C01308864704740F28801C2F20001F5
:1003D000C86C0130C864704740F28801C2F2000165
:1003E000086D01300865704740F28801C2F20001D3
:1003F000486D01304865704740F28801C2F2000143
:10040000486A01304862704740F28801C2F2000138
:10041000886A01308862704740F28801C2F20001A8
:10042000C8680130C860704740F28801C2F200011C
:10043000486C01304864704740F28801C2F2000104
:10044000C86A0130C862704740F28801C2F20001F8
:10045000486B01304863704740F28801C2F20001E6
:10046000C86B0130C863704740F28801C2F20001D6
:10047000086B01300863704740F28801C2F2000146
:10048000886B01308863704740F28801C2F2000136
:10049000086C01300864704780B590B0DDF848C042
:1004A000CDF83CC00E930D920C910B90002004905F
:1004B000042107918DF8280008900C9A019962F3A5
:1004C0001C0101919DF8071001F0F7018DF807104C
:1004D0009DF8061001F0F00108318DF80610FF219B
:1004E0008DF800108DF80100BDF80010ADF8041073
:1004F000019921F060410691099040F6EC00C2F2AA
:100500000000006805A902AA04AB00F037F810B09B
:1005100080BD00007047000081B0EFF3108072B61C
:100520000090FFE7FEE7000084B00290019102987E
:1005300090F820008DF803009DF80300012805D0F5
:10054000FFE79DF8030002280AD1FFE7019A02980D
:10055000016848691043486100208DF80F0008E0E9
:100560000299486A40F48020486201208DF80F000B
:10057000FFE79DF80F0004B07047000088B00690B8
:10058000059104920393069890F820008DF80700D7
:1005900006980068806800900598806808B9FFE7B1
:1005A00000E0FFE79DF80700012806D0FFE79DF86F
:1005B0000700022840F08080FFE79DF80300400715
:1005C00000280CD4FFE79DF803000007002806D49C
:1005D000FFE79DF80300C006002864D5FFE70098F8
:1005E000C0F30160029002990120884003990860DD
:1005F0000598806868B9FFE705980168C06840EA17
:10060000415006990968029A01EB0211C1F8800174
:100610000EE005994A688868C96840EAC200084344
:1006200006990968029A01EB0211C1F88001FFE7FF
:100630000598006906990968029A01EB0211C1F850
:1006400084010598007D01280CD1FFE70698006819
:10065000029900EB0111D1F8840140F48070C1F8D7
:100660008401FFE70498406806990968029A01EB43
:100670000211C1F88C010498006806990968029A71
:1006800001EB0211C1F8880106980068029900EB9D
:100690000111D1F8800140F00100C1F88001002073
:1006A0008DF81F0011E00699486A40F40010486276
:1006B00001208DF81F0008E00699486A40F4802068
:1006C000486201208DF81F00FFE79DF81F0008B069
:1006D0007047000086B00490039104980068019070
:1006E000049890F820008DF803009DF8030001287D
:1006F00006D0FFE79DF80300022840F09B80FFE74B
:100700000199D1F8000240F00100C1F800020398FD
:10071000406900F01F01012088400290029A01996F
:10072000D1F81C029043C1F81C020398C069F0B9CB
:10073000FFE7029A0199D1F80C029043C1F80C022C
:10074000039A9088D168526940EA0140019901EB0F
:10075000C201C1F84002039A10889168526940EAC8
:100760000140019901EBC201C1F84402FFE703987F
:10077000C06901281ED1FFE7029A0199D1F80C0245
:100780001043C1F80C02039A90881168526940EA3C
:100790000140019901EBC201C1F84002039A90891E
:1007A0009168526940EA0140019901EBC201C1F828
:1007B0004402FFE70398806940B9FFE7029A019974
:1007C000D1F804029043C1F8040207E0029A0199AB
:1007D000D1F804021043C1F80402FFE7039800694E
:1007E00040B9FFE7029A0199D1F814029043C1F889
:1007F000140207E0029A0199D1F814021043C1F8DB
:100800001402FFE70398006A012808D1FFE7029A63
:100810000199D1F81C021043C1F81C02FFE70199AD
:10082000D1F8000220F00100C1F8000200208DF88C
:10083000170008E00499486A40F4802048620120CB
:100840008DF81700FFE79DF8170006B0704700000D
:1008500080B582B001900198406A08B9FFE7C4E012
:100860000198406AC00718B1FFE7FFF795FDFFE761
:100870000198406A8007002803D5FFE7FFF784FD51
:10088000FFE70198406A4007002803D5FFE7FFF71C
:1008900063FDFFE70198406A0007002803D5FFE7E2
:1008A000FFF7BAFDFFE70198406AC006002803D5AC
:1008B000FFE7FFF779FDFFE70198406A800600280F
:1008C00003D5FFE7FFF738FDFFE70198406A4006D0
:1008D000002803D5FFE7FFF747FDFFE70198406ACF
:1008E0000006002803D5FFE7FFF72EFDFFE701987C
:1008F000406AC005002803D5FFE7FFF73DFDFFE78D
:100900000198406A8005002803D5FFE7FFF774FDD2
:10091000FFE70198406A4005002803D5FFE7FFF78D
:1009200073FDFFE70198406A0005002803D5FFE743
:10093000FFF782FDFFE70198406AC004002803D555
:10094000FFE7FFF791FDFFE70198406A8004002868
:1009500003D5FFE7FFF778FDFFE70198406A400401
:10096000002803D5FFE7FFF787FDFFE70198406AFE
:100970000004002803D5FFE7FFF76EFDFFE70198AD
:10098000406AC003002803D5FFE7FFF77DFDFFE7BE
:100990000198406A8003002803D5FFE7FFF744FD74
:1009A000FFE70198406A4003002803D5FFE7FFF7FF
:1009B00003FDFFE70198406A0003002803D5FFE725
:1009C000FFF702FDFFE70198406AC002002803D547
:1009D000FFE7FFF701FDFFE70198406A800200286A
:1009E00003D5FFE7FFF700FDFFE702B080BD000081
:1009F00086B00490039102920193049890F820002D
:100A00008DF803009DF80300012806D0FFE79DF84C
:100A10000300022840F0E880FFE7039880B9FFE771
:100A200004980068C068800748B9FFE70499486ADD
:100A300040F40010486201208DF81700DDE00FE05F
:100A4000049800680069800748B9FFE70499486A7C
:100A500040F40010486201208DF81700CDE0FFE758
:100A600004980068039900EB0110D0F8B00100F081
:100A70000400029988600298806858B9FFE70498DA
:100A80000068039900EB0110D0F8B001400D029905
:100A900008600AE004980068039900EB0110D0F8A0
:100AA000B001C00802994860FFE704980068039904
:100AB00000EB0110D0F8B00100F002000299C8600C
:100AC00004980068039900EB0110D0F8B40100F01D
:100AD0000F00082804D3FFE70299082008610BE003
:100AE00004980068039900EB0110D0F8B40100F0FD
:100AF0000F0002990861FFE704980068039900EB72
:100B00000110D0F8B40180B2000A029988610498FB
:100B10000068039900EB0110D0F8B401000C0299B1
:100B2000486104980068039900EB0110D0F8B801FF
:100B30000199087004980068039900EB0110D0F83F
:100B4000B801000A0199487004980068039900EB05
:100B50000110D0F8B801000C019988700498006861
:100B6000039900EB0110D0F8B801000E0199C8708C
:100B700004980068039900EB0110D0F8BC010199BA
:100B8000087104980068039900EB0110D0F8BC01CB
:100B9000000A0199487104980068039900EB01105C
:100BA000D0F8BC01000C0199887104980068039981
:100BB00000EB0110D0F8BC01000E0199C871039838
:100BC00038B9FFE704980168C86840F02000C860A1
:100BD00006E004980168086940F020000861FFE71A
:100BE00000208DF8170008E00499486A40F480203E
:100BF000486201208DF81700FFE79DF8170006B046
:100C00007047000080B58AB00990002008900998CC
:100C10000068406907900998006840680690099844
:100C200000688068059009980068C0680490099879
:100C300000680069039009980068806902909DF837
:100C40001C00C007002800F09480FFE79DF8140006
:100C5000C00758B3FFE709980168012088609DF834
:100C600014008007002804D5FFE70998816A8847A7
:100C70001BE09DF814004007002805D5FFE7089801
:100C800040F4006008900FE09DF814000007002871
:100C900005D5FFE7089840F48050089003E00998D4
:100CA000416B8847FFE7FFE7FFE7FFE79DF8150087
:100CB000C00760B3FFE7099801684FF4807088604F
:100CC0009DF815008007002804D5FFE70998C16A40
:100CD00088471BE09DF815004007002805D5FFE771
:100CE000089840F4005008900FE09DF815000007A8
:100CF000002805D5FFE7089840F48040089003E0FD
:100D00000998816B8847FFE7FFE7FFE7FFE79DF85A
:100D10001600C00760B3FFE7099801684FF4803000
:100D200088609DF816008007002804D5FFE7099821
:100D3000016B88471BE09DF816004007002805D589
:100D4000FFE7089840F4004008900FE09DF8160077
:100D50000007002805D5FFE7089840F48030089088
:100D600003E00998C16B8847FFE7FFE7FFE7FFE76C
:100D7000FFE79DF81C000007002810D5FFE79DF84D
:100D80001000C006002809D5FFE7089840F400705D
:100D90000890099801681020C860FFE7FFE79DF8F8
:100DA0001C00400700280FD5FFE79DF81000000742
:100DB000002808D5FFE7099801680820C86009984D
:100DC000416C8847FFE7FFE79DF81C00800700287B
:100DD0000BD5FFE709980068C068800720B1FFE7DE
:100DE0000998016C8847FFE7FFE79DF81C00400663
:100DF000002810D5FFE79DF80C00C006002809D593
:100E0000FFE7089840F48060089009980168102076
:100E10000861FFE7FFE79DF81C00800600280FD55A
:100E2000FFE79DF80C000007002808D5FFE70998A8
:100E30000168082008610998C16C8847FFE7FFE74F
:100E40009DF81C00C00600280BD5FFE70998006834
:100E50000069800720B1FFE70998816C8847FFE7A8
:100E6000FFE79DF81E00800700280FD5FFE79DF8DB
:100E70001800C006002808D5FFE70998016810206F
:100E800048600998016D8847FFE7FFE79DF81E005D
:100E9000C00778B1FFE79DF818000007002808D5C3
:100EA000FFE709980168082048600998416D884764
:100EB000FFE7FFE79DF81D000006002840F18D8048
:100EC000FFE79DF818004007002840F18180FFE708
:100ED0009DF81D00C00750B1FFE79DF80800C0074E
:100EE00028B1FFE7089840F001000890FFE79DF85F
:100EF0001D00800700280BD5FFE79DF8080080073C
:100F0000002805D5FFE7089840F002000890FFE7A9
:100F10009DF81D00400700280BD5FFE79DF808004D
:100F20004007002805D5FFE7089840F00400089026
:100F3000FFE79DF81D000007002848D5FFE79DF852
:100F4000080010F0700F42D0FFE7029800F0700028
:100F500001460191102814D0FFE70198202815D0F0
:100F6000FFE70198302816D0FFE70198402817D0F6
:100F7000FFE70198502818D0FFE70198602819D0A2
:100F80001DE0089840F00800089019E0089840F02B
:100F90001000089014E0089840F0200008900FE03E
:100FA000089840F0400008900AE0089840F080005F
:100FB000089005E0089840F48070089000E0FFE792
:100FC00009980168886920F070008861FFE7FFE7F1
:100FD0000998016804204860FFE7089848B1FFE7D6
:100FE000089A0999486A104348620998816D8847B0
:100FF000FFE70AB080BD000080B584B0029002987F
:1010000020B9FFE701208DF80F003AE1029890F82F
:10101000200000285DD1FFE7029941F25150C0F64F
:1010200000000864029941F24950C0F6000048648B
:10103000029941F26150C0F600008864029941F2C1
:101040005950C0F60000C864029941F20560C0F62C
:1010500000008862029941F21560C0F60000C86283
:10106000029941F22560C0F600000863029941F23E
:10107000FD50C0F600004863029941F20D60C0F6D1
:1010800000008863029941F21D60C0F60000C86349
:10109000029941F26950C0F600000865029941F2D8
:1010A000F570C0F600004865029940F65100C0F6A0
:1010B000000088650298C06D38B9FFE7029941F2D7
:1010C000E520C0F60000C865FFE70298C16D8847BB
:1010D000FFE702980168086840F00100086000F02E
:1010E000EDFD0190FFE7029800684068C007A8B9CD
:1010F000FFE700F0E3FD0199401A0B280DD3FFE74D
:101100000299486A40F4003048620299052081F84B
:10111000200001208DF80F00B3E0E4E70298016899
:10112000086820F00200086000F0C8FD0190FFE7A9
:101130000298006840688007002815D5FFE700F096
:10114000BDFD0199401A0B280DD3FFE70299486AAB
:1011500040F4003048620299052081F82000012007
:101160008DF80F008DE0E3E70298007E012807D19B
:10117000FFE702980168086840F08000086006E018
:1011800002980168086820F080000860FFE7029874
:10119000407E012807D1FFE702980168086840F007
:1011A0004000086006E002980168086820F04000EE
:1011B0000860FFE70298807E012807D1FFE70298C8
:1011C0000168086840F02000086006E002980168A5
:1011D000086820F020000860FFE70298C07E012820
:1011E00007D1FFE702980168086820F01000086046
:1011F00006E002980168086840F010000860FFE708
:101200000298007F012807D1FFE70298016808686B
:1012100040F00800086006E002980168086820F0C5
:1012200008000860FFE70298407F012807D1FFE728
:1012300002980168086840F00400086006E002981F
:101240000168086820F004000860FFE7029B196845
:101250005A689868D3F80CC040EA0C00D3F810C064
:1012600040EA0C005B691843013A1043C8610299D7
:1012700000204862029A012182F820108DF80F00A8
:10128000FFE79DF80F0004B080BD000080B582B07C
:1012900001900198006846F20041C4F200018842C2
:1012A0001DD1FFE741F21C01C4F20201086820F0E1
:1012B0000070086040F60000C4F201004FF4C05115
:1012C00000F09CFA132000F07BFD142000F078FD64
:1012D000152000F075FD162000F072FDFFE702B04A
:1012E00080BD000080B58EB00D9000200C900B905A
:1012F0000A9009900D98006846F20041C4F200017E
:1013000088425ED1FFE7FFE741F21C00C4F2020011
:10131000016841F000710160006800F00070089001
:101320000898FFE7FFE741F21800C4F202000168E5
:1013300041F004010160006800F004000790079884
:10134000FFE74FF400600990002005900A900B9091
:1013500040F60000C4F20100009009A9019100F0DC
:101360001DFB009801994FF48052099202220A92C3
:1013700003220C9200F012FB059A132002901146F2
:1013800000F032FD029800F025FD059A142003902C
:10139000114600F029FD039800F01CFD059A152068
:1013A0000490114600F020FD049800F013FD059A0A
:1013B00016200690114600F017FD069800F00AFD71
:1013C000FFE70EB080BD000087B005908DF81310C8
:1013D000039200208DF80B00039848B9FFE70599A8
:1013E000486A40F48000486201208DF81B00A6E0A6
:1013F000059890F82000012870D1FFE79DF81300B0
:10140000014601910E285FD801990FF2080000EB08
:101410008100874600F01CB800F01EB800F020B82C
:1014200000F022B800F024B800F026B800F028B888
:1014300000F02AB800F02CB800F02EB800F030B858
:1014400000F032B800F034B800F036B800F038B828
:1014500003980599886240E003980599C8623CE0CA
:1014600003980599086338E003980599486334E0C8
:1014700003980599886330E003980599C8632CE0C8
:1014800003980599086428E003980599486424E0C6
:1014900003980599886420E003980599C8641CE0C6
:1014A00003980599086518E003980599486514E0C4
:1014B00003980599886510E003980599C8650CE0C4
:1014C00003980599086608E00599486A40F4800089
:1014D000486201208DF80B00FFE72BE0059890F89B
:1014E0002000E8B9FFE79DF81300014600910D28A0
:1014F00004D0FFE700980E2804D007E00398059970
:10150000C8650CE003980599086608E00599486AE3
:1015100040F48000486201208DF80B00FFE708E0EE
:101520000599486A40F48000486201208DF80B005C
:10153000FFE7FFE79DF80B008DF81B00FFE79DF824
:101540001B0007B07047000081B0009001B07047E9
:1015500081B0009001B0704781B0009001B0704739
:1015600081B0009001B0704781B0009001B0704729
:1015700080B584B00290029890F8200001282FD105
:10158000FFE70299022081F82000029801680868AC
:1015900020F00100086000F091FB0190FFE7029845
:1015A00000684068C007A8B1FFE700F087FB019919
:1015B000401A0B280DD3FFE70299486A40F4003027
:1015C00048620299052081F8200001208DF80F0063
:1015D0000FE0E4E70299002048628DF80F0008E070
:1015E0000299486A40F40020486201208DF80F00FB
:1015F000FFE79DF80F0004B080BD000081B00090AF
:1016000001B0704781B0009001B0704781B0009088
:1016100001B0704781B0009001B0704781B0009078
:1016200001B0704781B0009001B0704784B0039062
:101630008DF80B1000208DF80A00039890F8200018
:10164000012840F0A080FFE79DF80B0001460191C2
:101650000E2800F28E8001990FF2080000EB810045
:10166000874600BF00F01CB800F021B800F026B893
:1016700000F02BB800F030B800F035B800F03AB800
:1016800000F03FB800F044B800F049B800F04EB8A0
:1016900000F053B800F058B800F05DB800F062B840
:1016A000039941F20560C0F6000088626AE0039980
:1016B00041F21560C0F60000C86263E0039941F290
:1016C0002560C0F6000008635CE0039941F2FD501C
:1016D000C0F60000486355E0039941F20D60C0F682
:1016E000000088634EE0039941F21D60C0F60000DF
:1016F000C86347E0039941F25150C0F60000086406
:1017000040E0039941F24950C0F60000486439E0D6
:10171000039941F26150C0F60000886432E00399F9
:1017200041F25950C0F60000C8642BE0039941F221
:101730006950C0F60000086524E0039941F2F57095
:10174000C0F6000048651DE0039940F65100C0F660
:101750000000886516E0039941F2E520C0F600001C
:10176000C8650FE0039941F28D20C0F600000866BD
:1017700008E00399486A40F48000486201208DF82F
:101780000A00FFE731E0039890F8200018BBFFE75C
:101790009DF80B00014600910D2804D0FFE700984A
:1017A0000E2807D00DE0039941F2E520C0F60000B5
:1017B000C8650FE0039941F28D20C0F6000008666D
:1017C00008E00399486A40F48000486201208DF8DF
:1017D0000A00FFE708E00399486A40F48000486285
:1017E00001208DF80A00FFE7FFE79DF80A0004B02A
:1017F0007047000081B0009001B070478DB00C9030
:101800000B9100200A90FFE70B980A99C840002826
:1018100000F0C180FFE70B980A9A0121914008402F
:1018200009900998002800F0B280FFE70A9820F09C
:1018300003000821C4F20101405808900A9800F002
:10184000030081000F2000FA01F108980840089079
:10185000089805900C9840F60001C4F201018842F6
:1018600003D1FFE70020049026E00C9840F60041E9
:10187000C4F20101884203D1FFE70120039018E080
:101880000C9841F20001C4F20101884203D1FFE744
:10189000022002900AE00C9941F20042C4F20102D7
:1018A0000420914208BF03200290FFE702980390B2
:1018B000FFE703980490FFE7059804990A9A02F05D
:1018C000030292009140884232D1FFE7099A40F228
:1018D0000041C4F20101086890430860099A40F28F
:1018E0000441C4F20101086890430860099A40F27B
:1018F0000C41C4F20101086890430860099A40F263
:101900000841C4F201010868904308600A9800F099
:10191000030081000F2088400890089B0A9820F05F
:1019200003010822C4F20102885898438850FFE757
:101930000998FF2803D8FFE70C98019003E00C9862
:1019400004300190FFE7019807900998FF2804D818
:10195000FFE70A988000009006E00A996FF01F00E8
:1019600000EB81000090FFE7009806900798006860
:10197000069A0F219140884304219140084307991A
:101980000860099A0C99C8689043C860FFE70A98F4
:1019900001300A9038E70DB07047000090B00F900A
:1019A0000E9100200D900990FFE70E9800680D99A8
:1019B000C840002800F07F81FFE70D990120884092
:1019C0000C900E9800680C9908400B900B980C999D
:1019D000884240F06C81FFE70E984068059000282F
:1019E00051D0FFE7059801283AD0FFE70598022873
:1019F0003FD0FFE7059803285FD0FFE7059811283F
:101A000032D0FFE70598122838D0FFE7059800216B
:101A1000C1F21101884236D0FFE705980021C1F2DA
:101A2000120188422FD0FFE705980021C1F2210161
:101A3000884228D0FFE705980021C1F222018842A0
:101A400021D0FFE705980021C1F2310188421AD068
:101A5000FFE705980021C1F23201884213D02FE040
:101A60000E98C06809902CE00E98C0680430099068
:101A700027E00E98C0680830099022E00E98C068F0
:101A80000C3009901DE00E98806818B9FFE704201B
:101A9000099011E00E988068012806D1FFE7082020
:101AA00009900C980F99086105E0082009900C989E
:101AB0000F994861FFE7FFE703E00020099000E08D
:101AC000FFE70B98FF2803D8FFE70F98049003E087
:101AD0000F9804300490FFE7049808900B98FF28B3
:101AE00004D8FFE70D988000039006E00D996FF091
:101AF0001F0000EB81000390FFE703980790089810
:101B00000068079A0F219140884309999140084342
:101B1000089908600E98C079C006002840F1C68078
:101B2000FFE7FFE741F21800C4F20200016841F04C
:101B300001010160006800F0010006900698FFE7CF
:101B40000D9820F003000821C4F2010140580A90CA
:101B50000D9800F0030081000F2000FA01F10A98AF
:101B600088430A900F9840F60001C4F201018842B0
:101B700003D1FFE70020029026E00F9840F60041D5
:101B8000C4F20101884203D1FFE70120019018E06F
:101B90000F9841F20001C4F20101884203D1FFE72E
:101BA000022000900AE00F9941F20042C4F20102C3
:101BB0000420914208BF03200090FFE700980190A5
:101BC000FFE701980290FFE702980D9901F00301E9
:101BD000890000FA01F10A9808430A900A980D99C1
:101BE00021F003010822C4F2010288500E98807986
:101BF000C006002809D5FFE70B9A40F20841C4F25D
:101C0000010108681043086008E00B9A40F208419F
:101C1000C4F20101086890430860FFE70E988079DC
:101C20008006002809D5FFE70B9A40F20C41C4F268
:101C3000010108681043086008E00B9A40F20C416B
:101C4000C4F20101086890430860FFE70E988079AC
:101C50008007002809D5FFE70B9A40F20441C4F23F
:101C6000010108681043086008E00B9A40F2044143
:101C7000C4F20101086890430860FFE70E9880797C
:101C8000C00748B1FFE70B9A40F20041C4F20101DE
:101C900008681043086008E00B9A40F20041C4F263
:101CA0000101086890430860FFE7FFE7FFE70D9830
:101CB00001300D9079E610B07047000041F22840E5
:101CC000C2F200000068704740F21C00C2F200003F
:101CD000027841F22841C2F200010868104408600D
:101CE0007047000080B542F20001C4F202010868AA
:101CF00040F010000860032000F090F80F2000F082
:101D000005F800F03BF8002080BD000080B582B0EF
:101D1000009040F20400C2F20000006840F21C0192
:101D2000C2F200010A784FF47A71B1FBF2F1B0FB14
:101D3000F1F001F0BDFA20B1FFE701208DF80700B6
:101D400018E000980F280DD8FFE700994FF0FF30FA
:101D5000002200F049F8009840F22001C2F2000190
:101D6000086003E001208DF8070003E000208DF8F3
:101D70000700FFE79DF8070002B080BD82B0FFE7D3
:101D800041F21800C4F20200016841F00101016053
:101D9000006800F0010001900198FFE7FFE741F2C1
:101DA0001C00C4F20200016841F08051016000682B
:101DB00000F0805000900098FFE702B070470000EC
:101DC00080B582B08DF807009DF9070004F0F0F9A6
:101DD00002B080BD80B582B08DF807009DF9070084
:101DE00004F002FA02B080BD80B586B08DF817000D
:101DF000049103920020029004F00EFA02909DF9E3
:101E00001700019002980499039A02F017FA01460C
:101E1000019804F009FA06B080BD000080B582B0D8
:101E20000190019804F022FA02B080BD2021C4F292
:101E30000E2101200860704780B588B0079000200F
:101E40000690059004900390029007980190012855
:101E500066D0FFE70198022800F0A580FFE701980F
:101E6000102840F0B080FFE741F20400C4F2020005
:101E70000068039041F20000C4F202000068C00153
:101E800000284CD5FFE70398C0F3834146F2A43005
:101E9000C0F60000405C04909DF80E00C007F0B151
:101EA000FFE741F20400C4F202000068C0F34041C1
:101EB00046F2B430C0F60000405C06909DF80E007B
:101EC000C00758B1FFE7069941F20020C0F27A003E
:101ED000B0FBF1F0049948430590FFE707E0049850
:101EE00040F60011C0F23D0148430590FFE741F282
:101EF0000400C4F2020000684002002803D5FFE796
:101F0000059802900AE0059840004AF6AB21CAF60F
:101F1000AA21A0FB011040080290FFE7FFE753E071
:101F200041F22000C4F2020000680390039800F41C
:101F30004070B0F5807F0AD1FFE79DF80C00800764
:101F4000002804D5FFE74FF4004002902AE00398F0
:101F500000F44070B0F5007F0DD1FFE741F224009E
:101F6000C4F2020000688007002804D5FFE749F6A4
:101F70004040029015E0039800F44070B0F5407FB7
:101F80000DD1FFE741F20000C4F2020000688003B7
:101F9000002804D5FFE74FF22440029000E0FFE75D
:101FA000FFE7FFE710E000F029FA41F20401C4F274
:101FB0000201096801F44042022101EB5231B0FBF9
:101FC000F1F0029000E0FFE7029808B080BD000049
:101FD00080B586B0049000200390029004980078A9
:101FE000C007002800F0AC80FFE700208DF8070054
:101FF00041F21C00C4F202000068C000002813D4A3
:10200000FFE7FFE741F21C00C4F20200016841F063
:1020100080510160006800F0805000900098FFE758
:1020200001208DF80700FFE747F20000C4F200002E
:102030000068C005002822D4FFE747F20001C4F27F
:102040000001086840F480700860FFF737FE0390D5
:10205000FFE747F20000C4F200000068C005002856
:102060000CD4FFE7FFF72AFE0399401A652804D332
:10207000FFE703208DF817008AE0EAE7FFE741F267
:102080002000C4F20200006800F440700290029840
:10209000E0B3FFE702980499496801F4407188426F
:1020A00034D0FFE741F22001C4F20201086820F4B5
:1020B0004070029040F24042C4F24222012010607F
:1020C00000201060029808609DF80800C007E0B189
:1020D000FFE7FFF7F3FD0390FFE741F22000C4F2B2
:1020E00002000068800700280ED4FFE7FFF7E6FD36
:1020F0000399401A41F28931884204D3FFE7032053
:102100008DF8170044E0E8E7FFE7FFE741F2200120
:10211000C4F20201086820F44070049A5268104327
:1021200008609DF80700012809D1FFE741F21C0172
:10213000C4F20201086820F080500860FFE7FFE762
:1021400004980078800700280CD5FFE741F20401CD
:10215000C4F20201086820F44040049A92681043D7
:102160000860FFE704980078C00600280CD5FFE758
:1021700041F20401C4F20201086820F48000049ACC
:10218000D26810430860FFE700208DF81700FFE7D2
:102190009DF8170006B080BD80B584B00290019113
:1021A000029820B9FFE701208DF80F001BE101988C
:1021B00042F20001C4F20201096801F007018842FD
:1021C00016D9FFE742F20000C4F20200016821F0D4
:1021D0000701019A11430160006800F007000199AE
:1021E000884204D0FFE701208DF80F00FBE0FFE7F5
:1021F00002980078800700282AD5FFE70298007827
:102200004007002809D5FFE741F20401C4F20201AA
:10221000086840F4E0600860FFE702980078000773
:10222000002809D5FFE741F20401C4F20201086861
:1022300040F460500860FFE741F20401C4F202017B
:10224000086820F0F000029A926810430860FFE7E7
:1022500002980078C007002860D0FFE70298406825
:1022600001280ED1FFE741F20000C4F2020000682D
:102270008003002804D4FFE701208DF80F00B2E0AE
:1022800021E00298406802280ED1FFE741F20000E9
:10229000C4F2020000688001002804D4FFE7012096
:1022A0008DF80F009FE00DE041F20000C4F2020043
:1022B00000688007002804D4FFE701208DF80F0094
:1022C00091E0FFE7FFE741F20401C4F20201086870
:1022D00020F00300029A526810430860FFF7EEFCFA
:1022E0000090FFE741F20400C4F20200006800F031
:1022F0000C0002994968B0EB810F0ED0FFE7FFF7A1
:10230000DDFC0099401A41F28931884204D3FFE78D
:1023100003208DF80F0066E0E4E7FFE7019842F242
:102320000001C4F20201096801F00701884216D2D7
:10233000FFE742F20000C4F20200016821F0070149
:10234000019A11430160006800F00700019988427A
:1023500004D0FFE701208DF80F0044E0FFE702986A
:102360000078400700280CD5FFE741F20401C4F2D1
:102370000201086820F4E060029AD2681043086005
:10238000FFE702980078000700280DD5FFE741F22B
:102390000401C4F20201086820F46050029A126934
:1023A00040EAC2000860FFE700F03AF841F2040199
:1023B000C4F202010968C9B20A0946F28C31C0F6BA
:1023C0000001895CC84040F20401C2F200010860CB
:1023D00040F22000C2F200000068FFF797FC0020E6
:1023E0008DF80F00FFE79DF80F0004B080BD0000DE
:1023F00040F20400C2F200000068704780B5FFF7A9
:10240000F7FF41F20401C4F202010968C1F3C222DC
:1024100046F29C31C0F60001895CC84080BD0000D6
:1024200086B000200590049003900290019041F244
:102430000400C4F2020000680590059800F00C004A
:102440000146009100283FD0FFE70098042804D0FF
:10245000FFE70098082806D037E041F20020C0F2DC
:102460007A00019037E00598C0F3834146F2B63018
:10247000C0F60000405C02909DF81600C007C0B195
:10248000FFE741F20400C4F202000068C0F34041DB
:1024900046F2C630C0F60000405C0490029841F25B
:1024A0000021C0F27A0148430499B0FBF1F0039097
:1024B00007E0029840F60011C0F23D014843039046
:1024C000FFE70398019006E0FFE741F20020C0F229
:1024D0007A000190FFE7019806B0704780B588B098
:1024E00007900691059200200490039002900190BD
:1024F000022102910321049103904FF48070019016
:10250000FFE741F21800C4F20200016841F0040143
:102510000160006800F0040000900098FFE740F6BA
:102520000000C4F2010001A9FFF738FA41F20401EA
:10253000C4F20201086820F0E060069A10430860C7
:1025400008B080BD80B586B00490049820B9FFE73C
:1025500001208DF817002EE304980078C0070028AA
:1025600000F0AE80FFE741F20400C4F20200006810
:1025700000F00C00042813D0FFE741F20400C4F27D
:102580000200006800F00C0008281BD1FFE741F2B0
:102590000400C4F202000068C003002812D5FFE75F
:1025A00041F20000C4F2020000688003002808D550
:1025B000FFE70498406820B9FFE701208DF8170075
:1025C000F9E27CE0FFE704984068B0F5803F09D16C
:1025D000FFE741F20001C4F20201086840F48030D4
:1025E000086032E00498406868B9FFE741F20001F2
:1025F000C4F20201086820F480300860086820F402
:102600008020086020E004984068B0F5A02F0DD12C
:10261000FFE741F20001C4F20201086840F48020A3
:102620000860086840F4803008600CE041F2000166
:10263000C4F20201086820F480300860086820F4C1
:1026400080200860FFE7FFE7FFE7FFE704984068A6
:10265000D0B1FFE7FFF732FB0390FFE741F2000044
:10266000C4F202000068800300280CD4FFE7FFF7E3
:1026700025FB0399401A652804D3FFE703208DF852
:10268000170098E2EAE719E0FFF718FB0390FFE76D
:1026900041F20000C4F202000068800300280CD55B
:1026A000FFE7FFF70BFB0399401A652804D3FFE708
:1026B00003208DF817007EE2EAE7FFE7FFE7FFE778
:1026C000049800788007002840F18D80FFE741F2F0
:1026D0000400C4F20200006810F00C0F13D0FFE7F2
:1026E00041F20400C4F20200006800F00C00082867
:1026F00029D1FFE741F20400C4F202000068C003E0
:10270000002820D4FFE741F20000C4F20200006874
:102710008007002809D5FFE704980069012804D044
:10272000FFE701208DF8170045E241F20001C4F2F5
:102730000201086820F0F800049A526940EAC200D9
:102740000860FFE74EE00498006958B3FFE70021F6
:10275000C4F2422101200860FFF7B0FA0390FFE7BE
:1027600041F20000C4F202000068800700280CD487
:10277000FFE7FFF7A3FA0399401A032804D3FFE702
:1027800003208DF8170016E2EAE741F20001C4F2D7
:102790000201086820F0F800049A526940EAC20079
:1027A00008601EE00021C4F2422100200860FFF70B
:1027B00085FA0390FFE741F20000C4F202000068CE
:1027C000800700280CD5FFE7FFF778FA0399401A35
:1027D000032804D3FFE703208DF81700EBE1EAE7B5
:1027E000FFE7FFE7FFE7049800780007002848D5D7
:1027F000FFE70498806918B3FFE740F28041C4F214
:10280000422101200860FFF759FA0390FFE741F2E7
:102810002400C4F202000068800700280CD4FFE7FF
:10282000FFF74CFA0399401A032804D3FFE703206B
:102830008DF81700BFE1EAE7012002F0ABFF1FE0CF
:1028400040F28041C4F2422100200860FFF736FACE
:102850000390FFE741F22400C4F202000068800701
:1028600000280CD5FFE7FFF729FA0399401A03283F
:1028700004D3FFE703208DF817009CE1EAE7FFE7A8
:10288000FFE7049800784007002840F1D880FFE770
:1028900000208DF8070041F21C00C4F2020000681D
:1028A000C000002813D4FFE7FFE741F21C00C4F288
:1028B0000200016841F080510160006800F0805022
:1028C00000900098FFE701208DF80700FFE747F22E
:1028D0000000C4F200000068C005002822D4FFE711
:1028E00047F20001C4F20001086840F480700860FB
:1028F000FFF7E4F90390FFE747F20000C4F200009D
:102900000068C00500280CD4FFE7FFF7D7F903994A
:10291000401A652804D3FFE703208DF817004AE129
:10292000EAE7FFE7FFE70498C068012809D1FFE75D
:1029300041F22001C4F20201086840F00100086081
:1029400031E00498C06868B9FFE741F22001C4F2A1
:102950000201086820F001000860086820F0040007
:1029600008601FE00498C06805280DD1FFE741F218
:102970002001C4F20201086840F004000860086801
:1029800040F0010008600CE041F22001C4F20201B5
:10299000086820F001000860086820F00400086062
:1029A000FFE7FFE7FFE7FFE70498C068E0B1FFE754
:1029B000FFF784F90390FFE741F22000C4F2020020
:1029C0000068800700280ED4FFE7FFF777F9039926
:1029D000401A41F28931884204D3FFE703208DF881
:1029E0001700E8E0E8E71BE0FFF768F90390FFE76E
:1029F00041F22000C4F202000068800700280ED5D2
:102A0000FFE7FFF75BF90399401A41F289318842E9
:102A100004D3FFE703208DF81700CCE0E8E7FFE7D9
:102A20009DF80700012809D1FFE741F21C01C4F21B
:102A30000201086820F080500860FFE7FFE7049873
:102A4000C069002800F0B380FFE741F20400C4F23F
:102A50000200006800F00C00082800F08280FFE708
:102A60000498C06902285CD1FFE76021C4F24221CA
:102A700000200860FFF722F90390FFE741F2000011
:102A8000C4F202000068800100280CD5FFE7FFF7C0
:102A900015F90399401A032804D3FFE703208DF8A2
:102AA000170088E0EAE70498006AB0F5803F0CD18F
:102AB000FFE741F20401C4F20201086820F400308B
:102AC000049A926810430860FFE741F20401C4F2DF
:102AD0000201086820F47410049B1A6A5B6A1A43A6
:102AE000104308606021C4F2422101200860FFF712
:102AF000E5F80390FFE741F20000C4F2020000682D
:102B0000800100280CD4FFE7FFF7D8F80399401A9A
:102B1000032804D3FFE703208DF817004BE0EAE712
:102B20001EE06021C4F2422100200860FFF7C6F8D1
:102B30000390FFE741F20000C4F202000068800148
:102B400000280CD5FFE7FFF7B9F80399401A0328CE
:102B500004D3FFE703208DF817002CE0EAE7FFE736
:102B600024E00498C069012804D1FFE701208DF812
:102B7000170020E041F20400C4F202000068029055
:102B8000029800F480300499096A884208D1FFE76E
:102B9000029800F470100499496A884204D0FFE753
:102BA00001208DF8170006E0FFE7FFE7FFE70020B0
:102BB0008DF81700FFE79DF8170006B080BD0000F4
:102BC00080B586B004900391029200208DF8060033
:102BD000ADF80400049818B1FFE7039820B9FFE7A7
:102BE00001208DF8170034E0049801A9002200F0BC
:102BF00035F820B1FFE701208DF8170029E004988F
:102C0000007B039908700498C07B0399C8700498EE
:102C1000407B039948700498807B039988700298E0
:102C200098B1FFE70398C07802F0E8FD0399C870F7
:102C30000398407802F0E2FD039948700398807889
:102C400002F0DCFD03998870FFE700208DF8170083
:102C5000FFE79DF8170006B080BD000080B588B082
:102C6000069005910492002003900290019000903C
:102C7000069818B1FFE7059820B9FFE701208DF805
:102C80001F00C0E00698006840684007002803D590
:102C9000FFE7012018B906E0012020B9FFE7012075
:102CA0008DF81F00AFE0069802F02EFF0390039905
:102CB0004BF2C530C9F2A210A1FB0021C90A009154
:102CC000039BA3FB0021C90A4FF4616201FB12338D
:102CD00048F68901C8F68801A3FB01C35B09DDF84A
:102CE00014C08CF80130039BA3FB00C0C00A00FB9A
:102CF0001230A0FB011251090901A1EB5211A0EB06
:102D0000810005998870009818285ED3FFE7009825
:102D10004AF6AB21CAF6AA21A0FB012000090190C6
:102D20000098A0FB0121090901EB4101A0EBC100C2
:102D300005990870069802F0CDFE029002980130C5
:102D400050B1FFE702980399884205D9FFE703993C
:102D50000298401A029003E04FF0FF300290FFE724
:102D6000019840F2A32141430398A0EBC1100390C6
:102D70000698039902F098FF20B1FFE701208DF833
:102D80001F0040E00298013078B1FFE703990298F4
:102D9000084402900698029902F05EFF20B1FFE716
:102DA00001208DF81F002EE00AE00698029902F03B
:102DB00053FF20B1FFE701208DF81F0023E0FFE75C
:102DC0000698019902F038FD03E000980599087013
:102DD000FFE7049898B1FFE70598007802F00EFD30
:102DE000059908700598407802F008FD059948702B
:102DF0000598807802F002FD05998870FFE70020B1
:102E00008DF81F00FFE79DF81F0008B080BD00008F
:102E100080B584B0029000200190029820B9FFE7AD
:102E200001208DF80F0084E00298407C38B9FFE75C
:102E3000029900200874029800F080F8FFE70299D8
:102E400002204874029800F001FA38B1FFE70299B5
:102E50000420487401208DF80F006AE0029802F007
:102E6000A5FD38B1FFE702990420487401208DF8D0
:102E70000F005EE002980168486820F00700486093
:102E80000298806848B1FFE746F63041C4F200017D
:102E9000086820F001000860FFE746F62C41C4F204
:102EA0000001086820F46070029A9268104308607C
:102EB00002984068013020B1FFE702984068019015
:102EC00012E00120FEF7B8FF0190019838B9FFE742
:102ED00002990420487401208DF80F0029E0019820
:102EE00001380190FFE7FFE7BDF8060000F00F0092
:102EF000029909688860BDF8040002990968C860F1
:102F0000029802F07FFD38B1FFE70299042048746F
:102F100001208DF80F000CE002990020C873029A7E
:102F200001215173029A9173029A51748DF80F0026
:102F3000FFE79DF80F0004B080BD000080B582B0AF
:102F400001900198006842F60001C4F20001884235
:102F500018D1FFE7FEF76AFFFFE741F21C00C4F259
:102F60000200016841F000610160006800F000604B
:102F700000900098FFE740F23C41C4F2422101205A
:102F80000860FFE702B080BD80B588B0069005916B
:102F900004920020039002900190069818B1FFE778
:102FA000059820B9FFE701208DF81F00A7E0FFE793
:102FB0000698007C012804D1FFE702208DF81F004D
:102FC0009DE0069901200874FFE7FFE706990220BB
:102FD0004874049868B9FFE70598C0780699C873E3
:102FE0000598407806994873059880780699887303
:102FF00012E00598C07802F0EBFB0699C8730598BB
:10300000407802F0E5FB069948730598807802F055
:10301000DFFB06998873FFE70698417B827BC07BC4
:1030200002F0A8FD069908730698007B05990870C0
:10303000069802F069FD039003984BF2C531C9F27E
:10304000A211A0FB0110C00A0190019819284AD3CF
:10305000FFE701984AF6AB21CAF6AA21A0FB0110AE
:10306000000940F2A32141430398A0EBC110039053
:103070000698039902F018FE60B1FFE70699042054
:103080004874FFE7069900200874FFE701208DF8D7
:103090001F0034E0069802F01DFD029002980130F6
:1030A00000B3FFE70298039988421AD2FFE702981B
:1030B00045F28011C0F2010108440290069802997D
:1030C00002F0CAFD60B1FFE7069904204874FFE7EB
:1030D000069900200874FFE701208DF81F000EE01C
:1030E000FFE7FFE7FFE7069901204874FFE706992D
:1030F00000200874FFE700208DF81F00FFE79DF80F
:103100001F0008B080BD000080B588B00690059112
:103110000492002003900290069818B1FFE70598EA
:1031200020B9FFE701208DF81F008AE0FFE706982D
:10313000007C012804D1FFE702208DF81F0080E009
:10314000069901200874FFE7FFE7069902204874FA
:10315000049870B9FFE7059908784A7889784FF4A0
:1031600061635843C2EB021200EB820008440390F3
:103170001BE00598007802F02BFB4FF46161484397
:1031800000900598407802F023FB01460098C1EBBF
:10319000011100EB810001900598807802F018FB86
:1031A0000146019808440390FFE70698039902F04E
:1031B0007BFD60B1FFE7069904204874FFE706999C
:1031C00000200874FFE701208DF81F0039E0069801
:1031D0000168486820F005004860069802F07AFC13
:1031E00002900298013000B3FFE7029803998842E9
:1031F0001AD2FFE7029845F28011C0F2010108449B
:1032000002900698029902F027FD60B1FFE7069947
:1032100004204874FFE7069900200874FFE70120A6
:103220008DF81F000DE0FFE7FFE7069901204874C5
:10323000FFE7069900200874FFE700208DF81F00C3
:10324000FFE79DF81F0008B080BD000080B584B086
:10325000029000200190029820B9FFE701208DF82C
:103260000F0021E002980168486820F008004860DB
:10327000FEF724FD0190FFE7029800684068000710
:1032800000280DD4FFE7FEF719FD0199401AB0F5AB
:103290007A7F04D9FFE703208DF80F0004E0EBE705
:1032A00000208DF80F00FFE79DF80F0004B080BDEF
:1032B00080B582B00190019802F020FD02B080BD7F
:1032C00081B0009001B0704781B0009001B07047AC
:1032D00081B0009001B0704781B0009001B070479C
:1032E00081B0009001B0704785B003900291FFE774
:1032F000039890F83C00012804D1FFE702208DF8E4
:1033000013005BE00399012081F83C00FFE7FFE731
:103310000399022081F83D000398006840680190FD
:103320000398006880680090019820F07000019078
:10333000029801680198084301900198039909686F
:1033400048600398006842F60041C4F201018842D7
:1033500018D0FFE703980068B0F1804F12D0FFE764
:103360000398006840F20041C4F20001884209D08D
:10337000FFE70398006840F60001C4F200018842AC
:103380000ED1FFE7009820F080000090029841687D
:103390000098084300900098039909688860FFE747
:1033A0000399012081F83D00FFE70399002081F88F
:1033B0003C00FFE700208DF81300FFE79DF81300A5
:1033C00005B0704780B582B00090009820B9FFE743
:1033D00001208DF807004DE0009890F83D00B0B94D
:1033E000FFE70099002081F83C00009802F0B4FD4E
:1033F0000098806C38B9FFE7009943F2B140C0F6FD
:1034000000008864FFE70098816C8847FFE7009917
:10341000022081F83D00009951F8040B02F0F4FC01
:103420000099012081F84600FFE70099012081F80A
:103430003E00009981F83F00009981F84000009912
:1034400081F84100FFE7FFE70099012081F8420081
:10345000009981F84300009981F84400009981F8AF
:103460004500FFE70099012081F83D0000208DF81C
:103470000700FFE79DF8070002B080BD80B582B06D
:1034800001900198006840F60001C4F200018842F2
:103490000CD1FFE741F21C01C4F20201086820F0E0
:1034A000040008601E20FEF78BFCFFE702B080BD21
:1034B00080B584B003900398006840F60001C4F220
:1034C0000001884219D1FFE7FFE741F21C00C4F276
:1034D0000200016841F004010160006800F004008E
:1034E00002900298FFE71E20019000221146FEF78D
:1034F0007BFC0198FEF76EFCFFE704B080BD000086
:1035000080B586B00490039100208DF80B00FFE792
:10351000049890F83C00012804D1FFE702208DF8C0
:103520001700ABE00499012081F83C00FFE7FFE7BA
:103530000499022081F83D00049800688068019099
:10354000019820F077000190019820F47F400190CD
:103550000198049909688860039800680090002821
:1035600072D0FFE7009810286ED0FFE7009820285F
:103570006AD0FFE70098302866D0FFE7009840281F
:1035800055D0FFE70098502837D0FFE70098602813
:1035900040D0FFE7009870280BD0FFE70098B0F507
:1035A000805F05D0FFE70098B0F5005F16D052E0CD
:1035B00055E004980068039B5A689968DB6802F03C
:1035C0009BFC0498006880680190019840F07700A7
:1035D0000190019804990968886040E004980068A7
:1035E000039B5A689968DB6802F086FC04980168BE
:1035F000886840F48040886031E004980068039A4D
:103600005168D26802F008FD04980068502102F069
:103610008DFC24E004980068039A5168D26802F097
:1036200023FD04980068602102F080FC17E00498F4
:103630000068039A5168D26802F0EEFC04980068B2
:10364000402102F073FC0AE00498006803990968BD
:1036500002F06CFC03E001208DF80B00FFE70499F9
:10366000012081F83D00FFE70499002081F83C002B
:10367000FFE79DF80B008DF81700FFE79DF8170096
:1036800006B080BD81B0009001B0704781B000905D
:1036900001B0704781B0009001B0704781B00090D8
:1036A00001B0704781B0009001B0704781B00090C8
:1036B00001B0704781B0009001B0704780B582B012
:1036C000019001980068006900F002010020B0EB51
:1036D000510F2BD0FFE701980068C06800F002018D
:1036E0000020B0EB510F20D0FFE7019801686FF088
:1036F000020008610199012008770198006880693B
:10370000800728B1FFE70198D0F89010884708E0BB
:103710000198D0F8981088470198D0F89C108847F5
:10372000FFE7019900200877FFE7FFE701980068AD
:10373000006900F004010020B0EB910F2CD0FFE7EE
:1037400001980068C06800F004010020B0EB910F00
:1037500021D0FFE7019801686FF00400086101992A
:103760000220087701980068806910F4407F05D036
:10377000FFE70198D0F89010884708E00198D0F84A
:10378000981088470198D0F89C108847FFE7019966
:1037900000200877FFE7FFE701980068006900F064
:1037A00008010020B0EBD10F2BD0FFE70198006893
:1037B000C06800F008010020B0EBD10F20D0FFE777
:1037C000019801686FF008000861019904200877EA
:1037D00001980068C069800728B1FFE70198D0F818
:1037E0009010884708E00198D0F898108847019811
:1037F000D0F89C108847FFE7019900200877FFE781
:10380000FFE701980068006900F010010020B0EBAC
:10381000111F2CD0FFE701980068C06800F010016C
:103820000020B0EB111F21D0FFE7019801686FF075
:103830001000086101990820087701980068C069A4
:1038400010F4407F05D0FFE70198D0F8901088472A
:1038500008E00198D0F8981088470198D0F89C109B
:103860008847FFE7019900200877FFE7FFE7019805
:1038700000680069C00788B1FFE701980068C06868
:10388000C00750B1FFE7019801686FF001000861BF
:103890000198D0F880108847FFE7FFE7019800689B
:1038A0000069C1B20020B0EBD11F14D0FFE701982E
:1038B0000068C068C1B20020B0EBD11F0AD0FFE79A
:1038C000019801686FF0800008610198D0F8B0108D
:1038D0008847FFE7FFE701980068006900F04001B2
:1038E0000020B0EB911F15D0FFE701980068C06879
:1038F00000F040010020B0EB911F0AD0FFE70198D3
:1039000001686FF0400008610198D0F8881088477E
:10391000FFE7FFE701980068006900F02001002040
:10392000B0EB511F15D0FFE701980068C06800F0A8
:1039300020010020B0EB511F0AD0FFE70198016879
:103940006FF0200008610198D0F8A8108847FFE7C1
:10395000FFE702B080BD000081B0009001B0704769
:1039600081B0009001B0704781B0009001B0704705
:1039700081B0009001B0704781B0009001B07047F5
:1039800081B0009001B0704781B0009001B07047E5
:1039900081B0009001B0704781B0009001B07047D5
:1039A00081B0009001B0704781B0009001B07047C5
:1039B00087B005908DF81310039200208DF80B004E
:1039C000039820B9FFE701208DF81B003DE1059821
:1039D00090F83D00012840F0C380FFE79DF81300F8
:1039E000014601911A2800F2B68001990FF20800F1
:1039F00000EB8100874600BF00F034B800F036B815
:103A000000F038B800F03AB800F03CB800F03EB82A
:103A100000F040B800F042B800F044B800F046B8FA
:103A200000F048B800F04AB800F04CB800F04EB8CA
:103A300000F050B800F053B800F056B800F059B894
:103A400000F05CB800F05FB800F062B800F065B854
:103A500000F068B800F06BB800F06EB800F071B814
:103A600000F074B803980599886478E00398059984
:103A7000C86474E003980599086570E00398059997
:103A800048656CE003980599886568E00398059996
:103A9000C86564E003980599086660E00398059995
:103AA00048665CE003980599886658E00398059994
:103AB000C86654E003980599086750E00398059993
:103AC00048674CE003980599886748E00398059992
:103AD000C86744E003980599C1F880003FE0039867
:103AE0000599C1F884003AE003980599C1F8880067
:103AF00035E003980599C1F88C0030E003980599EA
:103B0000C1F890002BE003980599C1F8940026E0D5
:103B100003980599C1F8980021E003980599C1F828
:103B20009C001CE003980599C1F8A00017E00398D9
:103B30000599C1F8A40012E003980599C1F8A800FE
:103B40000DE003980599C1F8AC0008E003980599C9
:103B5000C1F8B00003E001208DF80B00FFE76FE033
:103B6000059890F83D00002865D1FFE79DF8130007
:103B7000014600910D2859D800990FF2080000EB7A
:103B80008100874600F01AB800F01CB800F01EB89B
:103B900000F020B800F022B800F024B800F026B8F9
:103BA00000F028B800F02AB800F02CB800F02EB8C9
:103BB00000F030B800F032B800F034B8039805993E
:103BC000886437E003980599C86433E00398059941
:103BD00008652FE00398059948652BE0039805993F
:103BE000886527E003980599C86523E0039805993F
:103BF00008661FE00398059948661BE0039805993D
:103C0000886617E003980599C86613E0039805993C
:103C100008670FE00398059948670BE0039805993A
:103C2000886707E003980599C86703E001208DF8CD
:103C30000B00FFE703E001208DF80B00FFE7FFE733
:103C40009DF80B008DF81B00FFE79DF81B0007B0E7
:103C50007047000081B0009001B0704781B00090C3
:103C600001B0704784B003908DF80B1000208DF8E0
:103C70000A00039890F83D00012840F01481FFE706
:103C80009DF80B00014601911A2800F20781019965
:103C90000FF2080000EB8100874600BF00F034B847
:103CA00000F039B800F03EB800F043B800F048B872
:103CB00000F04DB800F052B800F057B800F05CB812
:103CC00000F061B800F066B800F06BB800F070B8B2
:103CD00000F075B800F07AB800F080B800F086B84F
:103CE00000F08CB800F092B800F098B800F09EB8E0
:103CF00000F0A4B800F0AAB800F0B0B800F0B6B870
:103D000000F0BCB800F0C2B8039943F2B140C0F66D
:103D100000008864C6E0039943F27D40C0F60000CD
:103D2000C864BFE0039943F2B560C0F600000865BF
:103D3000B8E0039943F2AD60C0F600004865B1E019
:103D4000039943F66910C0F600008865AAE003995C
:103D500043F66110C0F60000C865A3E0039943F67E
:103D60008910C0F6000008669CE0039943F68110B4
:103D7000C0F60000486695E0039943F67910C0F656
:103D8000000088668EE0039943F67110C0F60000CB
:103D9000C86687E0039943F28D60C0F600000867AB
:103DA00080E0039943F28560C0F60000486779E03F
:103DB000039943F2E120C0F60000886772E003999E
:103DC00043F2D920C0F60000C8676BE0039943F6C0
:103DD000A110C0F60000C1F8800063E0039943F62B
:103DE000A910C0F60000C1F884005BE0039943F617
:103DF0005540C0F60000C1F8880053E0039943F62F
:103E00005D40C0F60000C1F88C004BE0039943F21E
:103E10009D60C0F60000C1F8900043E0039943F2B2
:103E2000A560C0F60000C1F894003BE0039943F69A
:103E30005910C0F60000C1F8980033E0039943F62A
:103E40009110C0F60000C1F89C002BE0039943F6E6
:103E50009910C0F60000C1F8A00023E0039943F2D6
:103E60009560C0F60000C1F8A4001BE0039943F27E
:103E7000C920C0F60000C1F8A80013E0039943F27E
:103E8000D120C0F60000C1F8AC000BE0039943F26A
:103E9000C120C0F60000C1F8B00003E001208DF899
:103EA0000A00FFE79CE0039890F83D00002840F0EE
:103EB0009280FFE79DF80B00014600910D2800F26B
:103EC000858000990FF2080000EB8100874600BF53
:103ED00000F01AB800F01FB800F024B800F029B8BC
:103EE00000F02EB800F033B800F038B800F03DB85C
:103EF00000F042B800F047B800F04CB800F051B8FC
:103F000000F056B800F05BB8039943F2B140C0F638
:103F1000000088645EE0039943F27D40C0F6000033
:103F2000C86457E0039943F2B560C0F60000086525
:103F300050E0039943F2AD60C0F60000486549E0E7
:103F4000039943F66910C0F60000886542E00399C2
:103F500043F66110C0F60000C8653BE0039943F6E4
:103F60008910C0F60000086634E0039943F681101A
:103F7000C0F6000048662DE0039943F67910C0F6BC
:103F80000000886626E0039943F67110C0F6000031
:103F9000C8661FE0039943F28D60C0F60000086711
:103FA00018E0039943F28560C0F60000486711E00D
:103FB000039943F2E120C0F6000088670AE0039904
:103FC00043F2D920C0F60000C86703E001208DF855
:103FD0000A00FFE703E001208DF80A00FFE7FFE792
:103FE0009DF80A0004B07047FFE7FEE783B08DF844
:103FF0000B009DF80B0000F5FA608DF80B009DF8A2
:104000000B1001204BF65003C0F21E5345F6294217
:10401000CCF28F2201FB02314FEA31114DF20B72CB
:10402000C0F2A3029142019022D3FFE79DF80B104A
:10403000002089070090C1B9FFE79DF80B004BF6FF
:104040005002C0F21E5245F62941CCF28F2100FBEE
:1040500001204FEAB00145F62842C0F28F2200202D
:10406000914288BF01200090FFE700980190FFE790
:10407000019800F0010003B07047000080B582B0E5
:1040800040F6FC00C2F20000019046F20041C4F28A
:10409000000101600821416000228260C2604FF48B
:1040A000402101614FF48011416102760121417686
:1040B0008276C27602774177FCF79EFF18B1FFE760
:1040C000FCF72AFAFFE702B080BD000080B586B099
:1040D00000200590049003900290FFE741F2180041
:1040E000C4F20200016841F004010160006800F0C0
:1040F000040001900198FFE74FF4807002900220C5
:104100000390059040F60000C4F2010002A9FDF7FB
:1041100045FC06B080BD000080B582B000208DF85F
:104120000600ADF80400009040F66010C2F20000F6
:1041300042F60001C4F2000101604FF0FF3141601E
:104140004FF480718160FEF763FE18B1FFE7FCF762
:10415000E3F9FFE700208DF804008DF805008DF8E5
:10416000060040F66010C2F2000001A90122FEF72D
:10417000CBFF18B1FFE7FCF7CFF9FFE701228DF87D
:1041800000208DF801208DF8022000208DF803001A
:1041900040F66010C2F200006946FEF7F5FE18B165
:1041A000FFE7FCF7B9F9FFE702B080BD80B588B042
:1041B00000210191079106910591049103910291CB
:1041C00040F67410C2F2000040F60002C4F2000291
:1041D00002604FF6FF12426081604FF47A72C26053
:1041E00001618161FFF7EEF818B1FFE7FCF794F980
:1041F000FFE74FF48050049040F67410C2F20000C4
:1042000004A9FFF77DF918B1FFE7FCF785F9FFE78F
:1042100000200290039040F67410C2F2000002A940
:10422000FFF762F818B1FFE7FCF776F9FFE708B08F
:1042300080BD0000FFE7FEE7FFE7FEE788B00790DC
:1042400006910592079800F0070004900498C0F1C9
:104250000700052803D3FFE70420019004E0049839
:10426000C0F107000190FFE7019803900498043023
:10427000062803D8FFE70020009003E004980338E5
:104280000090FFE70098029006980399012202FA35
:1042900001F101390840029B984005999A40013A82
:1042A0001140084308B0704780B58AB0DDF830C0CF
:1042B000CDF820C00793069205910490BDF8140034
:1042C000ADF80C00BDF80C00000B0146029104286B
:1042D00056D802990FF2080000EB8100874600BF14
:1042E00000F008B800F014B800F020B800F02CB8C6
:1042F00000F038B804980599069A079BDDF820C0AD
:10430000EE46CEF800C000F07FFE8DF827003BE0BF
:1043100004980599069A079BDDF820C0EE46CEF872
:1043200000C000F0A7FD8DF827002DE00498059946
:10433000069A079BDDF820C0EE46CEF800C000F0DC
:10434000DDFD8DF827001FE004980599069A079B6C
:10435000DDF820C0EE46CEF800C000F07FFC8DF8FE
:10436000270011E004980599069A079BDDF820C004
:10437000EE46CEF800C000F0F7FC8DF8270003E011
:1043800001208DF82700FFE79DF827000AB080BDC7
:1043900080B58AB0DDF830C0CDF820C00793069212
:1043A00005910490BDF81400ADF80C00BDF80C00A8
:1043B000000901460291032840D802990FF2080033
:1043C00000EB8100874600BF00F006B800F012B88D
:1043D00000F01CB800F026B804980599069A079BCF
:1043E000DDF820C0EE46CEF800C000F003FF8DF8E7
:1043F00027002BE004980599069A079BDDF820C05A
:10440000EE46CEF800C000F03FFE1BE00498059990
:10441000069A079BDDF820C0EE46CEF800C000F0FB
:104420004BFE0FE004980599069A079BDDF820C023
:10443000EE46CEF800C000F089FE03E001208DF8C2
:10444000270003E000208DF82700FFE79DF82700F4
:104450000AB080BD80B58EB08DF837000C910B92FC
:104460009DF83700069000210791012008900591E2
:1044700009900E200A900C98C0F34F3001900C98D0
:10448000C000043080B202900B98C0F34F3003900C
:104490000B98C000043080B2049040F6EC00C2F2E9
:1044A0000000006801A9FCF715F918B1FFE7FCF757
:1044B00033F8FFE70EB080BD80B582B08DF80700FD
:1044C0009DF80710481E009102280DD3FFE70098C1
:1044D000032812D1FFE740F6F400C2F200000068A2
:1044E0000E21FFF7BFFBFFE740F6EC00C2F2000031
:1044F00000680621FDF79AF8FFE702B080BD0000D2
:1045000080B58AB0DDF830C0CDF820C007930692A0
:1045100005910490BDF81400ADF80C00BDF80C0036
:10452000000B01460291062868D802990FF2080094
:1045300000EB8100874600BF00F00CB800F016B811
:1045400000F020B800F02AB800F034B800F03EB80F
:1045500000F048B804980599069A079BDDF820C03A
:10456000EE46CEF800C000F0B3FE4BE0049805998B
:10457000069A079BDDF820C0EE46CEF800C000F09A
:10458000EFFE3FE004980599069A079BDDF820C0EE
:10459000EE46CEF800C000F0B3FE33E00498059973
:1045A000069A079BDDF820C0EE46CEF800C000F06A
:1045B000B3FE27E004980599069A079BDDF820C012
:1045C000EE46CEF800C000F0BFFE1BE0049805994F
:1045D000069A079BDDF820C0EE46CEF800C000F03A
:1045E00083FE0FE004980599069A079BDDF820C02A
:1045F000EE46CEF800C000F09BFE03E001208DF8EF
:10460000270003E000208DF82700FFE79DF8270032
:104610000AB080BD80B540F20800C2F20000016817
:1046200040F20C00C2F2000002680020FFF712FF07
:1046300040F6F800C2F20000016840F21000C2F239
:10464000000002680120FFF705FF40F21400C2F2EB
:104650000000016840F21800C2F200000268022067
:10466000FFF7F8FE80BD000080B592B0DDF850C0C5
:10467000CDF844C010930F920E910D90002006903B
:10468000042109918DF830000A900E9A039962F383
:104690001C0103919DF80F1001F0F7018DF80F1028
:1046A000039921F06041089108210B9147218DF871
:1046B000101041218DF8111053218DF812102D2169
:1046C0008DF813100290FFE7029803282CDCFFE717
:1046D000BDF83800029A0C21A1EB8201C84000F01D
:1046E0000F00019001980A2812D3FFE701984CF6B9
:1046F000CD41CCF6CC41A0FB0121C90801EB8101E1
:10470000A0EB41004130029904AA1144087106E06F
:1047100001983030029904AA11440871FFE7FFE7BD
:10472000029801300290CFE740F6EC00C2F20000A0
:10473000006807A904AA06ABFBF720FF12B080BDF2
:1047400080B586B0049003910292002001900498F5
:1047500078B1FFE7049940F6EC00C2F20000016076
:10476000006845F2BD62C0F600020621FCF72CFE8F
:1047700007E09DF80400FFF79FFE01208DF8170069
:1047800042E0019801300190039838B1FFE70398A7
:1047900040F6F001C2F20001086007E09DF8040055
:1047A000FFF78AFE02208DF817002DE001980130F6
:1047B0000190029878B1FFE7029940F6F400C2F246
:1047C00000000160006845F2E952C0F600020E21C7
:1047D000FFF7EEF807E09DF80400FFF76DFE0420F8
:1047E0008DF8170010E0019801300190FFF712FFDB
:1047F00040F2E001C2F20001087840F001000870C8
:1048000000208DF81700FFE79DF8170006B080BD67
:1048100080B582B0FFE7FBF76DFD002800F06781EF
:10482000FFE740F20000C2F20000007800EB8001D8
:1048300040F62820C2F2000000EB8100807900F0F1
:104840000F0002281DD1FFE740F20000C2F2000075
:10485000007800EB800140F62820C2F2000000EB57
:10486000810C50F82100DCF80410DCF80820DCF89A
:104870000C30DCF810C0EE46CEF800C0FFF714FD97
:104880002BE140F20000C2F20000007800EB800152
:1048900040F62820C2F2000000EB8100807900077A
:1048A000E8B9FFE740F20000C2F20000007800EB38
:1048B000800140F62820C2F2000000EB810C50F885
:1048C0002100DCF80410DCF80820DCF80C30DCF8FF
:1048D00010C0EE46CEF800C0FFF75AFDFCE040F2F3
:1048E0000000C2F20000007800EB800140F62820B2
:1048F000C2F2000000EB8100807900F00F00012877
:104900001DD1FFE740F20000C2F20000007800EB8A
:10491000800140F62820C2F2000000EB810C50F824
:104920002100DCF80410DCF80820DCF80C30DCF89E
:1049300010C0EE46CEF800C0FFF7E2FDCBE040F23B
:104940000000C2F20000007800EB800140F6282051
:10495000C2F2000000EB8100807900F00F00032814
:104960001DD1FFE740F20000C2F20000007800EB2A
:10497000800140F62820C2F2000000EB810C50F8C4
:104980002100DCF80410DCF80820DCF80C30DCF83E
:1049900010C0EE46CEF800C0FFF766FE9AE040F287
:1049A0000000C2F20000007800EB800140F62820F1
:1049B000C2F2000000EB8100807900F00F000428B3
:1049C00039D0FFE740F20000C2F20000007800EBAF
:1049D000800140F62820C2F2000000EB81008079BF
:1049E00000F00F00052826D0FFE740F20000C2F2D9
:1049F0000000007800EB800140F62820C2F20000A1
:104A000000EB8100807900F00F00062813D0FFE74B
:104A100040F20000C2F20000007800EB800140F696
:104A20002820C2F2000000EB8100807900F00F0026
:104A300007281DD1FFE740F20000C2F20000007815
:104A400000EB800140F62820C2F2000000EB810C50
:104A500050F82100DCF80410DCF80820DCF80C30F9
:104A6000DCF810C0EE46CEF800C000F041F830E0AF
:104A700040F20000C2F20000007800EB800140F636
:104A80002820C2F2000000EB8100807900F00F00C6
:104A900008281DD1FFE740F20000C2F200000078B4
:104AA00000EB800140F62820C2F2000000EB810CF0
:104AB00050F82100DCF80410DCF80820DCF80C3099
:104AC000DCF810C0EE46CEF800C0FBF7E5FCFFE7CF
:104AD000FFE7FFE7FFE7FFE7FFE740F20001C2F271
:104AE00000010878013000F07F000870FFE792E6CF
:104AF00080B588B0DDF828C0CDF818C005930492C1
:104B0000039102909DF80E0000F00F00043801465A
:104B10000191032846D801990FF2080000EB8100AB
:104B2000874600BF00F006B800F012B800F01EB8CB
:104B300000F02AB802980399049A059BDDF818C082
:104B4000EE46CEF800C000F017FC8DF81F002DE0F7
:104B500002980399049A059BDDF818C0EE46CEF83A
:104B600000C000F057FC8DF81F001FE00298039969
:104B7000049A059BDDF818C0EE46CEF800C000F0A0
:104B800097FC8DF81F0011E002980399049A059B89
:104B9000DDF818C0EE46CEF800C000F0D7FC8DF866
:104BA0001F0003E001208DF81F00FFE79DF81F00A4
:104BB00008B080BD80B584B0039040F6F000C2F22A
:104BC000000001680A68516841F01001516000223C
:104BD0008DF80A20ADF808200192039909788DF824
:104BE0000810039949788DF80910039989788DF890
:104BF0000A10006802A9FEF787FA18B1FFE7FBF771
:104C00008BFCFFE70398C0788DF8070003980079C4
:104C10008DF80500039840798DF806000398807997
:104C20008DF8040040F6F000C2F20000006801A90F
:104C30000022FEF7A9F918B1FFE7FBF76DFCFFE7CB
:104C400040F6F000C2F2000000680168486820F0F9
:104C50001000486004B080BD7047000080B590B07F
:104C6000DDF848C0CDF83CC00E930D920C910B902E
:104C700000200490042107918DF8280008900C99D9
:104C8000019861F31C0001909DF8070000F0F70007
:104C90008DF80700019820F06040069006200990EA
:104CA000BDF83000ADF8000049208DF80800532011
:104CB0008DF80900BDF800006FF31F3044F6D351A2
:104CC000C1F26201A0FB01012F2000EB91108DF8D1
:104CD0000A00BDF800006FF31F3048F21F51C5F203
:104CE000EB11A0FB0110400946F26761C6F2666154
:104CF00080FB012303F01C0202EB9302A0EB4200B5
:104D00002F308DF80B00BDF800006FF31F304CF60C
:104D1000CD42CCF6CC42A0FB0230C00880FB011390
:104D200003F0FC0101EB9301A0EB41002F308DF863
:104D30000C00BDF8000001466FF31F31A1FB0221FA
:104D4000C90801EB8101A0EB41002F308DF80D0067
:104D500040F6EC00C2F20000006805A902AA04AB0C
:104D6000FBF70CFC10B080BD80B590B0DDF848C0FA
:104D7000CDF83CC00E930D920C910B900020049046
:104D8000042107918DF8280008900C99019861F38F
:104D90001C0001909DF8070000F0F7008DF8070057
:104DA000019820F06040069006200990BDF8300080
:104DB000ADF8000054208DF8080053208DF809004C
:104DC000BDF800006FF31F3044F6D351C1F2620109
:104DD000A0FB01012F2000EB91108DF80A00BDF817
:104DE00000006FF31F3048F21F51C5F2EB11A0FB1A
:104DF0000110400946F26761C6F2666180FB01233B
:104E000003F01C0202EB9302A0EB42002F308DF85E
:104E10000B00BDF800006FF31F304CF6CD42CCF60E
:104E2000CC42A0FB0230C00880FB011303F0FC0160
:104E300001EB9301A0EB41002F308DF80C00BDF881
:104E4000000001466FF31F31A1FB0221C90801EBED
:104E50008101A0EB41002F308DF80D0040F6EC00F1
:104E6000C2F20000006805A902AA04ABFBF786FBAA
:104E700010B080BD80B590B0DDF848C0CDF83CC022
:104E80000E930D920C910B90002004900421079139
:104E90008DF8280008900C99019861F31C0001908E
:104EA0009DF8070000F0F7008DF80700019820F04A
:104EB000604006900720099055208DF80800532087
:104EC0008DF8090054208DF80A0041208DF80B0060
:104ED00056208DF80C004B208DF80D0049208DF8E0
:104EE0000E0040F6EC00C2F20000006805A902AA1C
:104EF00004ABFBF743FB10B080BD000080B590B061
:104F0000DDF848C0CDF83CC00E930D920C910B908B
:104F100000200490042107918DF8280008900C9936
:104F2000019861F31C0001909DF8070000F0F70064
:104F30008DF80700019820F0604006900620099047
:104F4000BDF83000ADF8000055208DF80800532062
:104F50008DF80900BDF800006FF31F3044F6D351FF
:104F6000C1F26201A0FB01012F2000EB91108DF82E
:104F70000A00BDF800006FF31F3048F21F51C5F260
:104F8000EB11A0FB0110400946F26761C6F26661B1
:104F900080FB012303F01C0202EB9302A0EB420012
:104FA0002F308DF80B00BDF800006FF31F304CF66A
:104FB000CD42CCF6CC42A0FB0230C00880FB0113EE
:104FC00003F0FC0101EB9301A0EB41002F308DF8C1
:104FD0000C00BDF8000001466FF31F31A1FB022158
:104FE000C90801EB8101A0EB41002F308DF80D00C5
:104FF00040F6EC00C2F20000006805A902AA04AB6A
:10500000FBF7BCFA10B080BD80B590B0DDF848C0A9
:10501000CDF83CC00E930D920C910B9000200490A3
:10502000042107918DF8280008900C99019861F3EC
:105030001C0001909DF8070000F0F7008DF80700B4
:10504000019820F0604006900620099055208DF8C8
:1050500008004E208DF8090049208DF80A005620DE
:105060008DF80B0045208DF80C0052208DF80D00B6
:1050700040F6EC00C2F20000006805A902AA04ABE9
:10508000FBF77CFA10B080BD80B585B0DDF81CC0A0
:10509000CDF810C0039302920191009040F2E0011C
:1050A000C2F2000108780122824300F0FE001044A1
:1050B000087005B080BD000080B58AB0DDF830C052
:1050C000CDF824C00893079206910590BDF81C0006
:1050D00008B9FFE737E0BDF81800ADF81000BDF8DB
:1050E000100000F00F00BDF81C10CA000221B1FB37
:1050F000F2F1884226D1FFE7002003900290019050
:10510000FFE70198BDF81C10884213DAFFE7019908
:1051100005A80844807AC90000FA01F202990398B0
:10512000891840EBE27002910390FFE7019801308B
:105130000190E6E702988008C00710B1FFE701F090
:10514000B3F8FFE7FFE70AB080BD000080B59EB06E
:10515000DDF880C0CDF874C01C931B921A91199091
:10516000BDF86C00082801DBFFE741E046F22C3176
:10517000C0F6000101A86022FBF726F89DF86E003A
:1051800017282EDCFFE79DF86F003B2829DCFFE79E
:105190009DF870003B2824DCFFE79DF87100632830
:1051A0001FDCFFE79DF872000C281ADCFFE79DF872
:1051B00071009DF873100091FEF718FF01460098EA
:1051C00001EB410201A901EB02119DF8722051F897
:1051D0002210884205DCFFE79DF87400072801DBF8
:1051E000FFE704E019A80A30FFF7E4FCFFE7FFE758
:1051F0001EB080BD80B594B0DDF858C0CDF84CC06D
:105200001293119210910F900022019208920420A3
:105210000B9007200D908DF838200C92109905986E
:1052200061F31C0005909DF8170000F0F7008DF861
:1052300017009DF8170000F0F80001308DF81700F6
:105240009DF81600022161F31F108DF816000598D5
:1052500020F060400A908DF81220ADF8102040F642
:10526000F000C2F200000290006804A9FDF7F6FC0D
:10527000019A02989DF810108DF818109DF81110E1
:105280008DF819109DF812108DF81A10039200680D
:1052900003A9FDF795FC9DF80F008DF81B009DF804
:1052A0000D008DF81C009DF80E008DF81D009DF876
:1052B0000C008DF81E0040F6EC00C2F20000006801
:1052C00009A906AA08ABFBF759F914B080BD000084
:1052D00080B585B0DDF81CC0CDF810C003930292F4
:1052E0000191009005B080BD80B585B0DDF81CC08F
:1052F000CDF810C0039302920191009005B080BDDB
:1053000080B585B0DDF81CC0CDF810C003930292C3
:105310000191009005B080BD80B585B0DDF81CC05E
:10532000CDF810C0039302920191009005B080BDAA
:1053300080B585B0DDF81CC0CDF810C00393029293
:105340000191009005B080BD80B586B0DDF820C029
:10535000CDF814C0049303920291019000F0A4FFD1
:1053600080B585B0DDF81CC0CDF810C00393029263
:105370000191009005B080BD80B590B0DDF848C0C7
:10538000CDF83CC00E930D920C910B900020049030
:10539000042107918DF8280008900C99019861F379
:1053A0001C0001909DF8070000F0F7008DF8070041
:1053B000019820F06040069008200990BDF8300068
:1053C000ADF800004D208DF8080043208DF809004D
:1053D00020218DF80A1053228DF80B20BDF80020F3
:1053E00012098DF80C208DF80D108DF80E009DF827
:1053F000000000F00F008DF80F0040F6EC00C2F244
:105400000000006805A902AA04ABFBF7B7F810B0CA
:1054100080BD000080B590B0DDF848C0CDF83CC03C
:105420000E930D920C910B90002004900421079193
:105430008DF8280008900C99019861F31C000190E8
:105440009DF8070000F0F7008DF80700019820F0A4
:105450006040069008200990BDF83000ADF80000CB
:105460004D208DF8080044208DF8090020208DF88B
:105470000A0053218DF80B10BDF8001009098DF8B2
:105480000C108DF80D0043208DF80E009DF80000E3
:1054900000F00F008DF80F0040F6EC00C2F20000A3
:1054A000006805A902AA04ABFBF768F810B080BD3C
:1054B00080B590B0DDF848C0CDF83CC00E930D9299
:1054C0000C910B9000200490042107918DF8280086
:1054D00008900C99019861F31C0001909DF8070059
:1054E00000F0F7008DF80700019820F0604006906A
:1054F00008200990BDF83000ADF800004D208DF86F
:10550000080048208DF8090020208DF80A0053215A
:105510008DF80B10BDF8001009098DF80C108DF8EE
:105520000D0043208DF80E009DF8000000F00F00E4
:105530008DF80F0040F6EC00C2F20000006805A9EB
:1055400002AA04ABFBF71AF810B080BD80B590B08A
:10555000DDF848C0CDF83CC00E930D920C910B9035
:1055600000200490042107918DF8280008900C99E0
:10557000019861F31C0001909DF8070000F0F7000E
:105580008DF80700019820F06040069008200990EF
:10559000BDF83000ADF800004D208DF8080049201E
:1055A0008DF8090020208DF80A0053218DF80B108A
:1055B000BDF8001009098DF80C108DF80D0043207E
:1055C0008DF80E009DF8000000F00F008DF80F0020
:1055D00040F6EC00C2F20000006805A902AA04AB84
:1055E000FAF7CCFF10B080BD80B58CB00B9040F2C4
:1055F000E000C2F200000078C00700285CD0FFE79E
:1056000000200490039901F060410391ADF80C0073
:105610009DF80E10022262F31F118DF80E109DF8F6
:105620000F1001F0F80101318DF80F109DF80E10E8
:1056300041F00F018DF80E109DF80F1001F0F701E9
:105640008DF80F109DF80F1041F010018DF80F101C
:10565000039921F060410691042107918DF82800FB
:1056600008900120099040F6E800C2F200000168AD
:1056700001310160039921F0604100910068B0F5AB
:10568000807F07D3FFE740F6E801C2F20001002067
:105690000860FFE740F6E800C2F2000000688DF8FD
:1056A000040040F6EC00C2F20000006805A901AA5F
:1056B00004ABFAF763FFFFE70CB080BD80B58EB096
:1056C0000D90FFE70D98002106AA04ABFBF790F9B7
:1056D00000285CD1FFE70898042857D1FFE740F67F
:1056E000E400C2F20000007840F20001C2F20001C2
:1056F0000978401A81300006002801D4FFE746E00F
:1057000040F6E400C2F200000078013000F07F00B3
:10571000ADF80E000799029861F31C0002909DF805
:105720000A0000F00F000F2820D1FFE79DF80A10B3
:105730009DF80B0000F0070240F2E400C2F2000006
:1057400000EB022201F0F003D15C41F00101D154E1
:105750009DF80A109DF80B2002F0070200EB0220D2
:1057600001F0F00101440020886010E00899099AD6
:105770000A9BBDF80EC00298EE46CEF804C00DF1AB
:10578000100CCEF800C000F099FCFFE79AE70EB0CD
:1057900080BD000082B00190019840F20401C2F285
:1057A00000010968C90844F6D352C1F26202A1FBA4
:1057B0000221890948430090FFE700BFFFE70098F6
:1057C000411E00910028F8D1FFE702B070470000A9
:1057D00082B08DF80700002000909DF807000009B6
:1057E00000EB80004000009000989DF8071001F049
:1057F0000F010844C0B202B07047000082B08DF8BB
:10580000070000200090FFE79DF807000A2809D351
:10581000FFE70098013000909DF807000A388DF8E6
:105820000700F1E7009800F00F019DF8070040EA3B
:10583000011002B07047000080B586B00590049159
:10584000002003900290019000900599C97B03917C
:105850000599497B02910599897B01910090FFE7A9
:1058600000980499884280F08C80FFE70298012814
:1058700018D0FFE70298032814D0FFE70298052804
:1058800010D0FFE7029807280CD0FFE702980828FD
:1058900008D0FFE702980A2804D0FFE702980C28F6
:1058A0001BD1FFE701981E2804D8FFE701980130BB
:1058B000019011E002980C2806D0FFE70298013011
:1058C00002900120019006E00120029001900398CF
:1058D00001300390FFE7FFE74EE0029804280CD068
:1058E000FFE70298062808D0FFE70298092804D0AD
:1058F000FFE702980B280FD1FFE701981D2804D875
:10590000FFE701980130019005E002980130029014
:1059100001200190FFE72EE0029802282AD1FFE73C
:1059200001981B2804D8FFE701980130019020E07E
:1059300001981C2811D1FFE7BDF80C0000F08EF88B
:1059400020B1FFE701980130019005E00298013095
:10595000029001200190FFE70AE001981D2806D17E
:10596000FFE702980130029001200190FFE7FFE776
:10597000FFE7FFE7FFE7FFE7FFE700980130009050
:105980006EE703980599C8730298059948730198C2
:105990000599887303989DF808109DF8042000F07D
:1059A000E9F80599087306B080BD000080B584B0A1
:1059B000029000200190FCF781F90190FFE7029826
:1059C00000684068800600280DD4FFE7FCF776F9F0
:1059D0000199401AB0F57A7F04D9FFE703208DF8CA
:1059E0000F000AE0EBE702980168486840F01000F9
:1059F000486000208DF80F00FFE79DF80F0004B00D
:105A000080BD000080B584B0029000200190029813
:105A10000168486820F010004860FCF74FF90190D9
:105A2000FFE7029800684068800600280DD4FFE771
:105A3000FCF744F90199401AB0F57A7F04D9FFE7E1
:105A400003208DF80F0004E0EBE700208DF80F0035
:105A5000FFE79DF80F0004B080BD000081B0ADF8F5
:105A60000000BDF80000800720B1FFE700208DF89E
:105A700003002BE0BDF8000045F62941CCF28F2150
:105A800048434FEAB00045F62941C0F28F218842D1
:105A900004D3FFE701208DF8030017E0BDF80000F4
:105AA00045F62941CCF28F2148434FEA30104DF2A0
:105AB0000A71C0F2A301884204D8FFE701208DF8E3
:105AC000030003E000208DF80300FFE79DF80300CA
:105AD00001B0704782B001900020ADF80200ADF82F
:105AE000000001980068006AADF8020001980068A3
:105AF000406AADF80000BDF80210BDF8000040EAB1
:105B0000014002B07047000084B003900020ADF85F
:105B10000A00ADF80800ADF8060000900398006890
:105B20008069ADF80A0003980068C069ADF8060006
:105B3000039800688069ADF80800BDF80A00BDF858
:105B4000081088420AD0FFE7BDF8081003980068E3
:105B5000C06980B240EA0140009007E0BDF80A1039
:105B6000BDF8060040EA01400090FFE7009804B04D
:105B70007047000084B003908DF80B108DF80A2058
:105B8000002001900090039800F5FA6001909DF8C4
:105B90000B0002282ED8FFE79DF80B001721484381
:105BA00048F63961C3F6E301A0FB01019DF80A0044
:105BB00000EB510001990844013900EB910048F2D3
:105BC0001F52C5F2EB12A1FB0221A0EB511000EB1A
:105BD000D110043044F62511C2F29241A0FB0121FC
:105BE000421A01EB52029108C900A1EB9201401A3E
:105BF00000902CE09DF80B001721484348F63961CE
:105C0000C3F6E301A0FB01019DF80A0000EB51007F
:105C10000199084400EB910048F21F52C5F2EB12C3
:105C2000A1FB0221A0EB511000EBD110023044F691
:105C30002511C2F29241A0FB0121421A01EB52024E
:105C40009108C900A1EB9201401A0090FFE79DF86E
:105C5000000004B07047000080B584B0039002914A
:105C600000208DF807000398FFF7A0FE20B1FFE7A2
:105C700001208DF8070013E0BDF80A0003990968B8
:105C80000862BDF808000399096848620398FFF7A5
:105C9000B9FE20B1FFE701208DF80700FFE7FFE71D
:105CA0009DF8070004B080BD80B584B003900291D8
:105CB00000208DF807000398FFF778FE20B1FFE77A
:105CC00001208DF8070013E0BDF80A000399096868
:105CD0008861BDF8080003990968C8610398FFF757
:105CE00091FE20B1FFE701208DF80700FFE7FFE7F5
:105CF0009DF8070004B080BD7047000080B582B0F9
:105D0000009000980138B0F1807F03D3FFE70120B5
:105D1000019019E0009801384EF21401CEF2000112
:105D200008604FF0FF300F2100F07EFA4EF21801AC
:105D3000CEF20001002008604EF21002CEF2000206
:105D4000072111600190FFE7019802B080BD0000BB
:105D500080B5FBF7B9FF80BD80B596B00CA8019067
:105D60002821FAF763FA0198002102910B910A9118
:105D700009910891079106910591049103910A22D6
:105D80000C9201221092102311931292022213926C
:105D900014914FF460111591FCF7D4FB18B1FFE793
:105DA000FAF7BAFBFFE70F200790022108910020C5
:105DB00009904FF480620A920B9007A8FCF7ECF967
:105DC00018B1FFE7FAF7A8FBFFE7012003904FF4B3
:105DD0000070049003A8FCF7FBF818B1FFE7FAF78E
:105DE0009BFBFFE74FF0E06100221046FCF776FBDB
:105DF00016B080BD7047000080B540F67410C2F246
:105E00000000FDF75BFC80BD83B002900191029819
:105E100000680090029842F60041C4F201018842F5
:105E200015D0FFE70298B0F1804F10D0FFE702983D
:105E300040F20041C4F20001884208D0FFE7029816
:105E400040F60001C4F2000188420AD1FFE7009841
:105E500020F070000090019841680098084300907D
:105E6000FFE7029842F60041C4F20101884215D0D2
:105E7000FFE70298B0F1804F10D0FFE7029840F2A0
:105E80000041C4F20001884208D0FFE7029840F6C2
:105E90000001C4F2000188420AD1FFE7009820F413
:105EA000407000900198C168009808430090FFE797
:105EB000009820F0800001994969084300900098FB
:105EC00002990860019880680299C8620198006888
:105ED00002998862029842F60041C4F201018842A8
:105EE00005D1FFE70198006902990863FFE702996D
:105EF0000120486103B0704785B00490039102927D
:105F00000193049880680090009820F47F400090EE
:105F100003980299019A41EA02210143009808433B
:105F2000009000980499886005B0704783B0029093
:105F30000191029880680090009820F07000009015
:105F400001980099084340F00700009000980299DA
:105F5000886003B07047000081B00090009943F65C
:105F6000A110C0F60000C1F88000009943F6A91006
:105F7000C0F60000C1F88400009943F65540C0F611
:105F80000000C1F88800009943F65D40C0F60000AB
:105F9000C1F88C00009943F29D60C0F60000C1F882
:105FA0009000009943F2A560C0F60000C1F894008B
:105FB000009943F65910C0F60000C1F89800009906
:105FC00043F69110C0F60000C1F89C00009943F61A
:105FD0009910C0F60000C1F8A000009943F2956046
:105FE000C0F60000C1F8A400009943F2C920C0F631
:105FF0000000C1F8A800009943F2D120C0F60000CB
:10600000C1F8AC00009943F2C120C0F60000C1F80D
:10601000B00001B07047000085B004900391029277
:106020000498006A00900499086A20F00100086250
:10603000049880690190019820F0F0000190029985
:10604000019840EA01100190009820F00A000090A9
:10605000039900980843009001980499886100987A
:106060000499086205B0704785B0049003910292CC
:106070000498006A00900499086A20F010000862F1
:10608000049880690190019820F470400190029971
:10609000019840EA01300190009820F0A0000090A3
:1060A0000399009840EA01100090019804998861D2
:1060B00000980499086205B07047000080B586B06A
:1060C00084460998DDF820E0CDF814C004910392CD
:1060D0000293ADF80600059BBDF8060000EB8000BA
:1060E00040F62821C2F2000101EB8002506863F300
:1060F0001C0050609DF81030BDF8060000EB8002D7
:1061000011F8220003F0010300F0FE00184401F82A
:1061100022009DF80C30BDF8060000EB800211F85B
:10612000220003F0010300F0FD0040EA430001F803
:1061300022000298BDF8062002EB820201EB8201E8
:10614000088100200090FFE700980299884214D24D
:10615000FFE70898009A805CBDF8061001EB810308
:1061600040F62821C2F2000101EB8301114488723C
:10617000FFE7009801300090E6E79DF8060040F642
:10618000E401C2F20001087006B080BD80B540F69F
:10619000FC00C2F20000FAF735FD80BD80B540F684
:1061A000FC00C2F20000FAF72DFD80BDFFE7FEE71C
:1061B00081B08DF803009DF90300002812D4FFE799
:1061C0009DF9031001F01F02012090404A094EF290
:1061D0008011CEF2000141F82200BFF34F8FBFF3D0
:1061E0006F8FFFE701B0704781B08DF803009DF914
:1061F000030000280ED4FFE79DF9031001F01F02F1
:10620000012090404A094EF20011CEF2000141F8FF
:106210002200FFE701B070474EF60C50CEF20000AE
:106220000068C0F30220704782B08DF8070000912B
:106230009DF9070000280AD4FFE7009800019DF9A6
:1062400007104EF20042CEF2000288540BE0009894
:1062500000019DF8071001F00F014EF61452CEF226
:1062600000028854FFE702B07047000083B002903C
:10627000029800F0070000904EF60C51CEF200019B
:106280000868019001984FF6FF02104001900198B4
:10629000009A40EA02200022C0F2FA521043019014
:1062A0000198086003B07047BFF34F8F4EF60C5152
:1062B000CEF20001086800F4E0600422C0F2FA5255
:1062C00010430860BFF34F8FFFE700BFFDE70000FA
:1062D00080B582B000200190FFF73EFDFBF702FD84
:1062E000FFF73AFDFDF7F2FEFDF7C8FEFDF714FFDC
:1062F000FDF75CFF40F6FC00C2F200000090FBF7E7
:1063000037F9009848F60241FAF70EF9009840F67E
:106310006011C2F2000140F67412C2F20002FEF7F0
:106320000FFAFEF775FAFFE7FEE700001F00000016
:106330001C0000001F0000001E0000001F000000E5
:106340001E0000001F0000001F0000001E000000D3
:106350001F0000001E0000001F0000001F000000C2
:106360001D0000001F0000001E0000001F000000B4
:106370001E0000001F0000001F0000001E000000A3
:106380001F0000001E0000001F00000000000000B1
:1063900000000000010203040607080900000000D5
:1063A0000102030402030405060708090A0B0C0D89
:1063B0000E0F1010010202030405060708090A0B5C
:1063C0000C0D0E0F10100102E86300080000002001
:1063D00028000000280100081064000828000020A0
:1063E000081A000044010008010000000024F40025
:1063F000000020090000F00F00000F0000000F0057
:1064000000000F000100000010000000000000006C
:04000005080000ED02
:00000001FF
